:1000000000308A00A52900000030A1001F08C33974
:1000100021049F000D30A000A00B0C289F149F18F6
:100020000F281E08A601A500260CA300250CA2007F
:10003000A30CA20CA30CA20CA30CA20C2208AB00D4
:100040000430A1001F08C33921049F000D30A00017
:10005000A00B28289F149F182B281E08A801A70072
:10006000280CA300270CA200A30CA20CA30CA20C2A
:10007000A30CA20C2208AC000C30A1001F08C3394D
:1000800021049F000D30A000A00B44289F149F184E
:1000900047281E08AA01A90000344C30840000083B
:1000A00003195F280230A100A001A00B5528A10B65
:1000B00054289730A000A00B5B28800B52280034F6
:1000C000CC014C08293C031C742805150830A000FD
:1000D000A00B6828000005110330A000A00B6E28BB
:1000E00000000000CC0A61280034CC014C08143C0C
:1000F000031C892805150830A000A00B7D280000EE
:1001000005110330A000A00B832800000000CC0ADA
:10011000762800340830CD02031C99284D30840025
:100120000310800C00080319992897280000800B01
:10013000962800340130B500B601B701B800B90007
:10014000C9010420051185122F0BA928BA01BB0192
:10015000AF28AF08031DAF28BA010130BB002B0840
:100160000F3C031DB5280E30AB00CB014B08033C00
:10017000031CD2280F30AB052B08B2000130B205AA
:10018000320BC9284B080A3C353E84000130800000
:10019000CE284B080A3C353E840080010310AB0C8E
:1001A000CB0AB628851DE1280B30CB004B080E3C4E
:1001B000031CE02835304B0784008001CB0AD62889
:1001C00007292C08053C031CF4280B30CB004B08F6
:1001D0000E3C031CF32835304B07840001308000AF
:1001E0008516CB0AE72807292C08093C031807299C
:1001F0000B30CB004B080D3C031C052935304B0759
:10020000840080018516CB0AFA280130C3002C082F
:10021000063C031C25290130C4002C08023C031CA9
:100220001529C5010130C60024292C08043C031CF3
:100230001D290130C500C60124292C08063C031CD9
:1002400024290130C500C6004029C4012C08083CFF
:10025000031C2D29C501C60140292C080A3C031C9A
:100260003529C5010130C60040292C080C3C031C6F
:100270003D290130C500C60140290130C500C60036
:10028000B1010330CB004B080F3C031C562935301D
:100290004B0784000310000DB10701304B07353EBA
:1002A00084000008B1070230CB074329460B5B29C5
:1002B0000310460DB1070330B105B108031D6429D1
:1002C0000130C700C8007829310B6A29C701013005
:1002D000C80078293108023C031D72290130C7008B
:1002E000C80178293108033C031D7829C701C801DA
:1002F000602075200130CB004B08143C031C98296A
:1003000035304B078400000B8E2960200330CC0071
:10031000C630CD008A20CC0B882996297520033061
:10032000CC00C630CD008A20CC0B9129CB0A7C2989
:100330000511AA08031DA1292908DB3C031CA129DA
:100340008516C830CC004D20F52984011F30830567
:100350001F1383161F149F141F159F150730831238
:100360009F00703083168F001B30650083121F13AF
:1003700083161F149F141F119F151F129F161F1302
:1003800083129F131F14703083168F0083128512FF
:100390000420A608031DD02925080C3C0318D429E5
:1003A000AF010330B000D8290130AF000230B000F7
:1003B000A608031DDF292508043C0318E1290420B1
:1003C000D829CA0130084A020318F0298516FA30E4
:1003D000CC004D208512FA30CC004D20CA0AE2290B
:0E03E0000130B400340BF6299A28F22963008C
:02400E00C43FAD
:00000001FF
